:1000000000308A004E2900000A108A100A11820767
:100010000A340D3458343D340034F701F801320805
:1000200003103318F707F70CF80CB318F707F70CA1
:10003000F80C3319F707F70CF80CB319F707F70C9E
:10004000F80C331AF707F70CF80CB31AF707F70C8C
:10005000F80C331BF707F70CF80CB31BF707F70C7A
:10006000F80C8B28B001AE010A30AF00AD01AC082E
:10007000031940283008B00A2C0784000008B1009A
:1000800031082D3C031D4D280130AE003008B00A68
:100090002C0784000008B100572831082B3C031DB1
:1000A00057283008B00A2C0784000008B100310836
:1000B0002F3C0318E6283108393C031CE628310898
:1000C000303C031D7A282C08300784000008783C57
:1000D000031971282C08300784000008583C031DC0
:1000E0007A281030AF00B00A3008B00A2C0784001C
:1000F0000008B1002F080A3C031D972831082F3C47
:10010000031896283108393C031C96280A30B2009F
:100110002D08B3000D28303031027807AD003008CB
:10012000B00A2C0784000008B1007E28E6282F08BA
:10013000103C031DE6283108603C0318A62831084E
:100140007A3C031CA6283108DF39A7283108B10002
:1001500031082F3C0318B0283108393C0318B8285F
:100160003108403C0318E6283108463C031CE628C9
:1001700031082F3C0318C9283108393C031CC92811
:100180002D0EB200F030B205303031023207AD0032
:10019000D2282D0EB200F030B205413031020A3EB5
:1001A0003207AD003008B00A2C0784000008B10007
:1001B0003108603C0318E32831087A3C031CE3282B
:1001C0003108DF39E4283108B100A8282E0BEE28C9
:1001D0002F080A3C031DEE28AD09AD0A2D08F800D2
:1001E00093292F08F8012E020318F9282E08F7008A
:1001F0000529F7010830B000AE0DF70D2F08770282
:100200000318F700F80DB00BFC2800342C08F70099
:10021000AC1B0E292D1D1A2920301329F709F70AC6
:100220007708AC002D30F80078080C1E15299900CD
:100230002D1DAD152C08AE006430AF00F1207708FD
:10024000AC0078083030031D2C292D183329AD1946
:1002500033292D1A20302E29AD112D12F8077808D8
:100260000C1E302999002C08AE000A30AF00F12096
:100270007708AC0078083030031D4229AD194729B2
:100280002D1A2030F80778080C1E442999003030C8
:10029000AC072C080C1E4A299900B62984011F308E
:1002A000830507309F00A0010130A100A201A30136
:1002B000A401CF3083169900223098009030831229
:1002C0009800AC012C080420AC0AF70077080C1E3B
:1002D0006729990004302C02031D6229A601260813
:1002E000043C031C8C292730260784008C1E7629A9
:1002F0001A08800027302607840000080D3C0319E7
:100300008C292730260784000008AC002C080C1E1E
:1003100087299900A60A6F292730260784008001C3
:100320002730AC0032287808A5000A300C1E962928
:1003300099000D300C1E9A29990027308400003056
:1003400000040319A9290C1EA32900089900840A96
:100350009F290A300C1EAA2999000D300C1EAE29C7
:1003600099002508AC001030AD0006290A300C1E9B
:10037000B72999000D300C1EBB2999006129630033
:02400E00693F08
:00000001FF
